:100F630000C000F900A400B000990092008200F8CC
:100F7300008000900088008300C600A10086008ED8
:0411B500135401FFCF
:0A11B900E51125E0F511EF421122C7
:0D11FB00E51125E0F511EFF4540142112239
:0412BC00EF521122BA
:0D109D00135401FD1211D17864E65401FFD7
:0710AA00EFF4540152112282
:0412C000EF421122C6
:07129300EFF45401421122A7
:0E11C300E511F45401FFE51154FE4FF5112221
:0E10B1001210D9AF30EFC4135401FF1212BC5D
:0610BF00E5115401FF22BF
:0D120800E511C313FFE51154015FF511223C
:0D121500E511C313FFE51154014FF511223F
:0E11D100E51125E0F511EDF45F540142112205
:0E11DF00E51125E0F511EFF45D5401421122F7
:100FA000121222AF24EFC4135401FFAE41EEC4135A
:030FB0005401FDEC
:080FB300EDF45F54015211221C
:08000300EFF45D5401521122DB
:08128300EDF45F540142112259
:08128B00EFF45D540142112251
:07129A00EDF45F5401FF2297
:0712A100EFF45D5401FF2290
:0D122200E51825E0FFE51154014FF51822F5
:0D122F00E5185401FFE51154FE4FF51122A2
:1010D900E5185401FFE51154FE4FF511E518C31346
:0310E900F51822D5
:101196008E5E8F5FE55F2DFFE55E3C8FF0020B6193
:1010EC008E5B8F5CC3E55C9DFFE55B9C8FF0020B18
:0110FC006192
:100FBB00900116E0FEA3E0FF7B017A0179167D100C
:020FCB007C00A8
:090FCD00120AA0EE8FF0020B6184
:0F11A6008B5B8A5C895D120AB2EE8FF0020B61DF
:06123C007B017A01791428
:07124200E475F001020B2925
:0712A80074FFF5F0020B29B1
:1010FD008E608F61E5605CFFE5615DCF8FF0020B67
:01110D006180
:100F1500900116E0FEA3E0FF900110E0FCA3E0FDC8
:060F25007B017A01791640
:100F2B008E5B8F5CE55B4CFFE55C4DCF8FF0020B6E
:010F3B006154
:10110E008E628F63E5626CFFE5636DCF8FF0020B2D
:01111E00616F
:10111F00EFF4FFEEF4FEEF2401FFE43E8FF0020B3D
:01112F00615E
:0612B600EFF45401FF22D9
:0E10C500900116E0FEA3E0FF7B017A00790C9B
:0610D300EE8FF0020B613C
:0A127900EFF4FFEEF48FF0020B61BA
:100EE6008B4B8A4C894D120AFEFFAEF0AB4EAA4FD1
:100EF600A950120AFEFDAB4BAA4CA94DE5F08DF0A8
:0F0F0600120B61AB4EAA4FA950EE8FF0020B6198
:100BD5008E518F528B538A5489557C037DE8120AB6
:100BE500B2EFC454F07B00FAAE51AF527C037DE8FE
:100BF500120AB28C518D52AE51AF527C007D6412F7
:100C05000AB2EFFEE4EE4202AE51AF527C007D64C3
:100C1500120AB28C518D52AE51AF527C007D0A1230
:100C25000AB2EFC4F8540FC868FFEEC454F048FE8A
:100C3500EFFBEE4202AE51AF527C007D0A120AB2C2
:100C45008C518D52E5514AFFE5524BAB53AA54A93D
:070C550055CF8FF0020B6187
:100CDB008E568F57E557780CCEA2E713CE13D8F864
:100CEB007E00540FFF7C037DE8120AA08E588F59AB
:100CFB00E556FF3395E07E00EF540FFF7C007D64DB
:100D0B00120AA0EF2559F559EE3558F558E557AEAF
:100D1B00567804CEA2E713CE13D8F87E00540FFFFB
:100D2B007C007D0A120AA0EF2559F559EE3558F5CE
:100D3B0058E557540F2559F559E43558F558855949
:040D4B00F0020B6146
:100FD600E51125E0F511C3EF9DEC6480F8EE648021
:0B0FE600984004431101225311FE2229
:100FF100E51125E0F511D3EF9DEC6480F8EE6480F6
:0B100100985004431101225311FE22FD
:10100C00E51125E0F511D3EF9DEC6480F8EE6480DA
:0B101C00984004431101225311FE22F2
:10102700E51125E0F511C3EF9DEC6480F8EE6480CF
:0B103700985004431101225311FE22C7
:10105C00E51125E0F511EF6D7002EE6C60044311A3
:06106C0001225311FE22D7
:10107200E51125E0F511EFB50508EEB504044311BD
:0610820001225311FE22C1
:0C0F8300900112E0FEA3E0FF7D0A7C005C
:100F8F00C3EF9DEC6480F8EE64809850035311FE1C
:010F9F00222F
:10113000D3EF9DEC6480F8EE64809840035311FE79
:01114000228C
:10114100D3EF9DEC6480F8EE64809850035311FE58
:01115100227B
:10115200C3EF9DEC6480F8EE64809840035311FE67
:01116200226A
:0C124900EFB50507EEB504035311FE22BB
:09108800E0FEA3E0FF74FFFDFC93
:0C109100EF6D7002EE6C60035311FE2244
:10116300C3EF9DEC6480F8EE648098400343110163
:011173002259
:10117400D3EF9DEC6480F8EE648098500343110132
:011184002248
:09104200E0FEA3E0FF7D097C0043
:10104B00D3EF9DEC6480F8EE64809840034311016C
:01105B002272
:10118500C3EF9DEC6480F8EE648098500343110131
:011195002237
:0C125500EF6D7002EE6C6003431101228B
:0C126100EFB50507EEB5040343110122B0
:0712AF00E4FF0FBF0AFC225F
:100EB600E4FEC2B41212AFC2B31212AFD2B3121210
:100EC600AFD2B41212AFE4FDEE25E0FE3094034338
:100ED6000601C2B31212AFD2B30DBD08EBAF0622A4
:1008BF000510E510C394054003E4F510E51014602E
:1008CF005B14700302097B1470030209C7240360D1
:1008DF0003020A197C0090000DE0540FFD25E0FF84
:1008EF00EC33FE74632FF582740F3EF583E493FCB3
:1008FF00740193FD43040890010AE0FFC41313131E
:10090F00540130E0057DFF020A6FEF131313541FDC
:10091F0020E003020A6F53057F020A6F90000CE07C
:10092F00FEA3E07804CEA2E713CE13D8F87C0054D0
:10093F000FFD25E0FFEC33FE74632FF582740F3E3D
:10094F00F583E493FC740193FD43040490010BE0E1
:10095F0030E0057DFF020A6F90010AE0FFC4540FDB
:10096F0020E003020A6F53057F020A6F90000CE02C
:10097F00FF3395E07C00EF540FFD25E0FFEC33FED5
:10098F0074632FF582740F3EF583E493FC74019327
:10099F00FD43040290010BE0FFC31330E0057DFF20
:1009AF00020A6F90010AE0FFC413540720E003020C
:1009BF000A6F53057F020A6F90000CE0FEA3E078E8
:1009CF000CCEA2E713CE13D8F87C00540FFD25E010
:1009DF00FFEC33FE74632FF582740F3EF583E493BF
:1009EF00FC740193FD43040190010BE0FF131354BA
:1009FF003F30E0047DFF806890010AE0FFC41313CD
:100A0F00540330E05B53057F805690010BE0F9C42F
:100A1F001313540175F008A4FBAAF0E9C4131313C0
:100A2F00540175F010A4FFE5F04AFAEF4BFBE9C44F
:100A3F0013540175F004A4FFEA45F0FAEB4FFBE9FC
:100A4F00C4540125E0FFE4334AFEEB4FFFE91313D3
:100A5F00135401FBEEEF4BF4FFEEF47410FCAD07F3
:100A6F007B10C2B31212AFEC20E704C2B78002D2E0
:100A7F00B71212AFED25E0FDEC33FCD2B31212AF7B
:100A8F00DBE0D2B71212AFC2B51212AFD2B502125B
:010A9F00AFA7
:1006D900E52E70030208BE152E0517E517B4051798
:1006E900AF30EFC4135401F45401FFC43354E0FF95
:1006F900E53054DF4FF530E517B40A1CAF30EFC4CD
:10070900135401F45401FFC43354E0FFE53054DFBE
:100719004FF530051DE4F517E4F55BE55B1313139D
:10072900541F2412F8E6FD7C00E55B5407FF7401B1
:100739007E00A807088005C333CE33CED8F9FFEE73
:100749005CFEEF5D4E6043E55B25E025E0246EF538
:1007590082E43400F583E0FEA3E0FFE55B25E025B4
:10076900E0246CF582E43400F583E0FCA3E0C39F48
:10077900EC9E5016E55B25E025E0246CF582E43417
:1007890000F583E475F001120AE8E55B25E025E050
:10079900246EF582E43400F583E0FEA3E0FFE55B17
:1007A90025E025E0246CF582E43400F583E0FCA320
:1007B900E0C39FEC9E407AE55B25E025E0246CF5DB
:1007C90082E43400FEC3E582946CFFEE9400FE7C63
:1007D900007D02120AB27C007D02120AB27C007D01
:1007E90008120AB2741E2FF8C000E6FFC007E55BC5
:1007F90025E025E0246CF582E43400FEC3E582940B
:100809006CFFEE9400FE7C007D02120AB27C007D32
:1008190002120AB27C007D08120AB2AF057401A85F
:1008290007088002C333D8FCFED0E04ED000F68022
:1008390079E55B25E025E0246CF582E43400FEC30C
:10084900E582946CFFEE9400FE7C007D02120AB2F0
:100859007C007D02120AB27C007D08120AB2741E65
:100869002FF8C000E6FFC007E55B25E025E0246C12
:10087900F582E43400FEC3E582946CFFEE9400FE39
:100889007C007D02120AB27C007D02120AB27C0051
:100899007D08120AB2AF057401A807088002C333A4
:1008A900D8FCF4FED0E05ED000F6055BE55B642081
:0608B90060030207242287
:100DFC00E51DB41E19AF30EFC413135401F45401A4
:100E0C00FFC4333354C0FFE53054BF4FF530E51DFC
:100E1C00B43C1CAF30EFC413135401F45401FFC4A1
:100E2C00333354C0FFE53054BF4FF530E4F51D2289
:03000B00020D4F94
:100D4F00C0E0C0D075D008758CEEAF30EF13131321
:100D5F005401F45401FF33333354F8FFE53054F7A3
:100D6F004FF530053AE53A30E0020516E53AB40A98
:100D7F0015AF30EFC45401F45401FFC454F0FFE534
:100D8F003054EF4FF530E53AB4141AAF30EFC45486
:100D9F0001F45401FFC454F0FFE53054EF4FF53028
:0A0DAF00052E753A00D0D0D0E032D6
:100DB9007594FF752F05E4F530F53190000CF0A31B
:100DC900F090010BE054F7F054EFF054DFF054BF0A
:100DD900F0547FF090010AE054F7F054EFF054DF3B
:100DE900F054BFF0547FF0A3E054FEF054FDF054EA
:030DF900FBF022EA
:0412C400752F092257
:100E3C00E4FFEF25E025E0246CF582E43400F58333
:100E4C00E4F0A3F00FBF20EAE4FF7F4090002CE415
:100E5C00F0A3DFFCE4FF741E2FF8E4F60FBF04F6DA
:0D0E6C00E4FF74192FF8E4F60FBF04F6221E
:0E11ED00758911D2B4D2B9D2A9D28CD2AF2258
:100E7900AFA0EFC3135455FEEF25E054AA4EFF135C
:100E8900135433FEEF25E025E054CC4EFF54F0FE19
:100E9900E590540F4EF4F522EF540FF4540FF52357
:0D0EA900120EB6EFF4F5248528800208BF74
:100C5C00E4FF74222FF8E6FE743F2FF8A6060FBFB0
:100C6C0006F0E4FF74282FF8E6FE74452FF8A6066C
:100C7C000FBF06F0E4FF74642FF8E6FE74202FF526
:100C8C0082E43401F583EEF00FBF20EAE4FF74EC4C
:100C9C002FF582E43400F583E0FE74402FF582E4F6
:100CAC003401F583EEF00FBF20E4E4FF741E2FF83F
:100CBC00E6FE74362FF8A6060FBF04F0E4FF741995
:0F0CCC002FF8E6FE74322FF8A6060FBF04F022B1
:100F3C00755A01120DB9120E3C1211ED120E7912E6
:100F4C00000E1206D9120DFC120C5CE55A60EDE491
:070F5C00F55A1212C480E5F2
:10000E00AF2FEF131211B5121222E51130E00F903F
:10001E00010CE0FEA3E0FF7D3B7C0012100CE5110D
:10002E0030E00690010E121042E51130E00F900103
:10003E0010E0FEA3E0FF7D057C0012104BE51130B1
:10004E00E006900112121042E51130E00F900114FB
:10005E00E0FEA3E0FF7D027C0012104B121208E5B9
:10006E001130E007E490010CF0A3F0E51130E00749
:10007E00E490010EF0A3F0E51130E007E4900110DA
:10008E00F0A3F0E51130E00D7B017A0179127F02C9
:10009E007E001210D3E51130E00D7B017A01791448
:1000AE007F017E001210D31210D9E51130E00790B7
:1000BE00010BE054F7F0E51130E00790010BE0542E
:1000CE00EFF0E51130E00790010BE054DFF0E511A1
:1000DE0030E00790010BE054BFF0E51130E00790DF
:1000EE00010BE0547FF0E51130E0067864E654FE33
:1000FE00F6E51130E0067864E654FDF6E51130E0E1
:10010E0007E4900000F0A3F0AF24EF131313540193
:10011E00FFAE41EE1313135401FD1211D1E5113050
:10012E00E0067864E64401F6E51130E0067864E610
:10013E0054FDF6AF24EFC413135401FFAE41EEC4C9
:10014E0013135401FD1211D17864E65401FF1212FB
:10015E00BCE51130E004E654FEF6E51130E007E4AC
:10016E0090010CF0A3F0AF24EFC41313135401FF4E
:10017E00AE41EEC4131312109DE51130E016E6FFEA
:10018E00C3135401FF1212B6EF5401FF25E0FFE630
:10019E0054FD4FF67864E65401FF1211B91210BFE8
:1001AE00EF5401FFC43333335480FF90010BE054FE
:1001BE007F4FF0121222AF24EFC45401FFAE41EE76
:1001CE00C45401FD120FB3E51130E0097B017A0032
:1001DE007900121242E51130E00F900000E0FEA30C
:1001EE00E0FF7D047C00120F8FE51130E007E490F4
:1001FE000000F0A3F012122FE51130E00E90000077
:10020E00E0FEA3E0FFE4FDFC121091120FA0E51139
:10021E0030E00312123CE51130E00F900114E0FEC5
:10022E00A3E0FF7D037C00120F8FE51130E007E4A1
:10023E00900114F0A3F012122FAF24EF13135401F8
:10024E00FFAE41EE13120FAFE51130E0097B017ADC
:10025E000179141212A8E51130E006900114121063
:10026E0088E51130E00D7B017A0179147F027E0062
:10027E001210D31210B1EF5401FF25E025E0FF90CC
:10028E00010BE054FB4FF012122FE51130E00F90EE
:10029E000000E0FEA3E0FF7D017C00121091120F22
:1002AE00A0E51130E0097B017A017912121242E5C4
:0102BE00112E
:1002BF0030E003120F83E51130E007E4900112F0F4
:1002CF00A3F012122FAF24EF13135401FFAE41EE20
:1002DF0013120FAFE51130E0097B017A0179121289
:1002EF0012A8E51130E006900112121088E51130C6
:1002FF00E00D7B017A0179127F097E001210D31273
:10030F0010B1EF5401FF25E0FF90010BE054FD4FBA
:10031F00F012122FE51130E00F900000E0FEA3E085
:10032F00FF7D027C00121091120FA0E51130E00941
:10033F007B017A017910121242E51130E00F900122
:10034F0010E0FEA3E0FF7D067C00120F8FE5113059
:10035F00E007E4900110F0A3F012122FAF24EF1377
:10036F00135401FFAE41EE13120FAFE51130E00948
:10037F007B017A0179101212A8E51130E006900185
:10038F0010121088E51130E00D7B017A0179107F92
:10039F00057E001210D31210B1EF5401FF90010B24
:1003AF00E054FE4FF01210D9E51130E00F9000002D
:1003BF00E0FEA3E0FF7D037C00121091120FA0E579
:1003CF001130E0097B017A01790E121242E51130EA
:1003DF00E00690010E120F86E51130E007E4900160
:1003EF000EF0A3F012122FAF24EF13135401FFAE30
:1003FF0041EE13120FAFE51130E0097B017A01795D
:10040F000E1212A8E51130E00690010E121088E5C9
:10041F001130E00D7B017A01790E7F097E001210F9
:10042F00D31210B1EF5401FFC43333335480FF9014
:10043F00010AE0547F4FF0AF30EFC41211B5121024
:10044F00BFEF5401FFC43354E0FFE054DF4FF0E03F
:10045F00FFC4135401FF90015EE0FEC412109DE52E
:10046F001130E0097B017A01790C1212421212222B
:10047F00E51130E00F90010CE0FEA3E0FF7D3C7C26
:10048F0000120F8FE51130E0097B017A01790E120E
:10049F001242E51130E007E490010CF0A3F01212C4
:1004AF002FE51130E00690010E120F86E51130E0B6
:1004BF00097B017A017910121242E51130E007E44D
:1004CF0090010EF0A3F012122FE51130E00F900102
:1004DF0010E0FEA3E0FF7D067C00120F8FE51130C8
:1004EF00E0097B017A017912121242E51130E0071F
:1004FF00E4900110F0A3F012122FE51130E0031277
:0A050F000F83E51130E00312123CE7
:10051900E51130E007E4900112F0A3F01210D9E5DB
:100529001130E00F900114E0FEA3E0FF7D027C0092
:10053900121072E51130E00F900112E0FEA3E0FF06
:100549007D047C00120F8FE51130E00F900114E05B
:10055900FEA3E0FF7D037C00121163121208E5116E
:1005690030E007E4900114F0A3F0E51130E007E46E
:10057900900112F0A3F0E52F5401FF1211B91212E4
:10058900227864E6FFC3135401FF1210AAE5113063
:10059900E00C7B017A017916E4FFFE1210D3E51114
:1005A90030E00E900116E0FEA3E0FF900114120F57
:1005B90020E51130E003120FBBE51130E00E900188
:1005C90016E0FEA3E0FF900112120F20E51130E0C2
:1005D90003120FBBE51130E003120F15E51130E0EE
:1005E90003120FBBE51130E00E900116E0FEA3E007
:1005F900FF90010E120F20E51130E0031210C51211
:1006090010D97864E6FFC3135401FF1212BCE51137
:1006190030E00C7B017A017916E4FFFE1210D3E574
:100629001130E003120F15E51130E003120FBBE59D
:100639001130E00E900116E0FEA3E0FF90010E12CA
:100649000F20E51130E003120FBBE51130E01590E2
:10065900010CE0FEA3E0FF7B017A0179187D0A7C99
:10066900001211A6E51130E00C900116E0FEA3E09E
:10067900FFA3120F20E51130E003120FBBE5113083
:10068900E015900118E0FEA3E0FF7B017A017918DB
:100699007D0A7C00120FCDE51130E01990010CE0C4
:1006A900FEA3E0FF900118E0FCA3E0FD7B017A01C5
:1006B90079181210ECE51130E00C900116E0FEA358
:1006C900E0FFA3120F20E51130E0031210C500224C
:0300000002126D7C
:0C126D00787FE4F6D8FD758183020F3C09
:100AA000EF8DF0A4A8F0CF8CF0A428CE8DF0A42E6A
:020AB000FE2224
:100AB200C2D5EC30E709B2D5E4C39DFDE49CFCEE5F
:100AC20030E715B2D5E4C39FFFE49EFE120B80C34C
:100AD200E49DFDE49CFC8003120B8030D507C3E447
:060AE2009FFFE49EFE22CE
:100AE800C5F0F8A3E028F0C5F0F8E5821582700299
:060AF8001583E038F02236
:100AFE00BB010A89828A83E0F5F0A3E022500687C3
:100B0E00F009E71922BBFE07E3F5F009E319228984
:0B0B1E00828A83E493F5F074019322B7
:100B2900BB010789828A83020AE8500B09C5F027AD
:100B3900F7C5F01937F722BBFE0D09F8E325F0F3E5
:100B4900C5F019E338F322F889828A837401932561
:080B5900F0C5F0F8E493382226
:100B6100BB010A89828A83F0E5F0A3F0225006F7DF
:0F0B710009A7F01922BBFE06F3E5F009F31922DC
:100B8000BC000BBE0029EF8DF084FFADF022E4CC59
:100B9000F875F008EF2FFFEE33FEEC33FCEE9DEC22
:100BA000984005FCEE9DFE0FD5F0E9E4CEFD22ED68
:100BB000F8F5F0EE8420D21CFEADF075F008EF2FB2
:100BC000FFED33FD4007985006D5F0F222C398FDA3
:050BD0000FD5F0EA2240
:00000001FF
